:200000000C94C8040C94E7040C94E7040C94E7040C94E7040C94E7040C94E7040C94E704A7
:200020000C94E7040C94E7040C94E7040C94E7040C94E7040C94E7040C94E7040C94E70468
:200040000C94E7040C94E7040C94E7040C94E7040C94FFFFFFFFFFFFFFFFFFFFFFFFFFFFE2
:20006000FFFFFFFFFFFFFFFFFFFFFFFFFFFFFFFFFFFF000000000000000000000000000092
:20008000000000000000000000000000000000000000000000000000000000000000000060
:2000A000000000000000000000000000000000000000000000000000000000000000000040
:2000C000000000000000000000000000000000000000000000000000000000000000000020
:2000E000000000000000000000000000000000000000000000000000000000000000000000
:020000040003F7
:020000040004F6
:00000001FF
